:0300000002000EED
:03000300020028D0
:20000B0002001F75810FD2AFD2A912002B80FE12001B80FB758CDC758A00050832050832F6
:20002B007400F50A748075F025C0E0C0F012013215811581120158749075F001F50C85F0B8
:20004B000DE50A4401F50A12011212011B1200621200BA02005222E50A540175F0007B0028
:20006B007C001201DD45F070030200B9E50C850DF01201C3F50C85F00D1201BAE50C850D8A
:20008B00F07B007C001201DD45F070030200A3E50904F509140200B9E50A54FEF50A74902E
:2000AB0075F001F50E85F00FE50A4402F50A22E50A540275F0007B007C001201DD45F070BC
:2000CB0003020111E50E850FF01201C3F50E85F00F1201BAE50E850FF07B007C001201DDFF
:2000EB0045F070030200FBE50914F50904020111E50A54FDF50A749075F001F50C85F00D0C
:20010B00E50A4401F50A22308DFDC28D438CDC22E509540779087A0275F00012017D898263
:20012B008A83E493F5902278FB12015B8603088604748075F0701201841201CA758921F53C
:20014B008DF58B75885975985222D2AF22C2AF22C82581C822C92581C97A0022D083D082A9
:20016B00CF2581F581CFC082C08322CF2581F581CF2229F9E5F03AFA22C002C001AAF0F9D4
:20018B007E007D007F11C3E933F9EA33FADF08F5F0E9D001D00222ED33FDEE33FEC3ED9BD9
:2001AB00F5F0EE9C40E0ADF0FED380DB1201BA04700205F0221201C314B4FF0215F02212AA
:2001CB0001C3F4C5F0F4C5F0221201E76009E4F5F0221201E760F7E4F5F00422C5F0C39C3A
:2001EB007003E5F09B22FBE493CB22FCE493FB740193CC22FAE493F9740193CA2280C0404E
:05020B0060203010909E
:00000001FF
